 Compare

 Timestamp is 56b152db (Wed Feb 03 04:07:39 2016)

 Preferred load address is 10000000

 Start         Length     Name                   Class
 0001:00000000 0000011cH .idata$5                CODE
 0001:0000011c 00000004H .CRT$XCA                CODE
 0001:00000120 00000004H .CRT$XCZ                CODE
 0001:00000124 00000004H .CRT$XIA                CODE
 0001:00000128 0000000cH .CRT$XIC                CODE
 0001:00000134 00000004H .CRT$XIZ                CODE
 0001:00000138 00000004H .CRT$XPA                CODE
 0001:0000013c 00000004H .CRT$XPZ                CODE
 0001:00000140 00000004H .CRT$XTA                CODE
 0001:00000144 00000004H .CRT$XTZ                CODE
 0001:00000148 00002280H .rdata                  CODE
 0001:000023c8 000000dcH .rdata$r                CODE
 0001:000024b0 0000000cH .rdata$sxdata           CODE
 0001:000024bc 00000004H .rtc$IAA                CODE
 0001:000024c0 00000004H .rtc$IZZ                CODE
 0001:000024c4 00000004H .rtc$TAA                CODE
 0001:000024c8 00000004H .rtc$TZZ                CODE
 0001:000024d0 0000793fH .text                   CODE
 0001:00009e0f 00000014H .text$yd                CODE
 0001:00009e28 0000021cH .xdata$x                CODE
 0001:0000a044 00000014H .idata$2                CODE
 0001:0000a058 00000014H .idata$3                CODE
 0001:0000a06c 0000011cH .idata$4                CODE
 0001:0000a188 000004f2H .idata$6                CODE
 0001:0000a680 00000090H .edata                  CODE
 0002:00000000 00000dc0H .data                   DATA
 0002:00000dc0 00000fc0H .bss                    DATA
 0003:00000000 00000058H .rsrc$01                DATA
 0003:00000060 00000380H .rsrc$02                DATA

  Address         Publics by Value              Rva+Base       Lib:Object

 0000:00000000       __except_list              00000000     <absolute>
 0000:00000003       ___safe_se_handler_count   00000003     <absolute>
 0000:00000000       ___ImageBase               10000000     <linker-defined>
 0001:00000000       __imp__lstrlenW@4          10001000     kernel32:KERNEL32.dll
 0001:00000004       __imp__ReadConsoleInputW@16 10001004     kernel32:KERNEL32.dll
 0001:00000008       __imp__PeekConsoleInputW@16 10001008     kernel32:KERNEL32.dll
 0001:0000000c       __imp__GetTickCount@0      1000100c     kernel32:KERNEL32.dll
 0001:00000010       __imp__lstrcatW@8          10001010     kernel32:KERNEL32.dll
 0001:00000014       __imp__lstrcpyW@8          10001014     kernel32:KERNEL32.dll
 0001:00000018       __imp__lstrcmpW@8          10001018     kernel32:KERNEL32.dll
 0001:0000001c       __imp__FindClose@4         1000101c     kernel32:KERNEL32.dll
 0001:00000020       __imp__FindNextFileW@8     10001020     kernel32:KERNEL32.dll
 0001:00000024       __imp__FindFirstFileW@8    10001024     kernel32:KERNEL32.dll
 0001:00000028       __imp__ReadFile@20         10001028     kernel32:KERNEL32.dll
 0001:0000002c       __imp__CloseHandle@4       1000102c     kernel32:KERNEL32.dll
 0001:00000030       __imp__CreateFileW@28      10001030     kernel32:KERNEL32.dll
 0001:00000034       __imp__SetConsoleTitleW@4  10001034     kernel32:KERNEL32.dll
 0001:00000038       __imp__GetConsoleTitleW@8  10001038     kernel32:KERNEL32.dll
 0001:0000003c       __imp__GetLastError@0      1000103c     kernel32:KERNEL32.dll
 0001:00000040       __imp__HeapReAlloc@16      10001040     kernel32:KERNEL32.dll
 0001:00000044       __imp__HeapFree@12         10001044     kernel32:KERNEL32.dll
 0001:00000048       __imp__HeapAlloc@12        10001048     kernel32:KERNEL32.dll
 0001:0000004c       __imp__GetCurrentThreadId@0 1000104c     kernel32:KERNEL32.dll
 0001:00000050       __imp__DecodePointer@4     10001050     kernel32:KERNEL32.dll
 0001:00000054       __imp__GetCommandLineA@0   10001054     kernel32:KERNEL32.dll
 0001:00000058       __imp__IsProcessorFeaturePresent@4 10001058     kernel32:KERNEL32.dll
 0001:0000005c       __imp__EncodePointer@4     1000105c     kernel32:KERNEL32.dll
 0001:00000060       __imp__HeapCreate@12       10001060     kernel32:KERNEL32.dll
 0001:00000064       __imp__HeapDestroy@4       10001064     kernel32:KERNEL32.dll
 0001:00000068       __imp__GetProcAddress@8    10001068     kernel32:KERNEL32.dll
 0001:0000006c       __imp__GetModuleHandleW@4  1000106c     kernel32:KERNEL32.dll
 0001:00000070       __imp__ExitProcess@4       10001070     kernel32:KERNEL32.dll
 0001:00000074       __imp__WriteFile@20        10001074     kernel32:KERNEL32.dll
 0001:00000078       __imp__GetStdHandle@4      10001078     kernel32:KERNEL32.dll
 0001:0000007c       __imp__GetModuleFileNameW@12 1000107c     kernel32:KERNEL32.dll
 0001:00000080       __imp__GetCPInfo@8         10001080     kernel32:KERNEL32.dll
 0001:00000084       __imp__InterlockedIncrement@4 10001084     kernel32:KERNEL32.dll
 0001:00000088       __imp__InterlockedDecrement@4 10001088     kernel32:KERNEL32.dll
 0001:0000008c       __imp__GetACP@0            1000108c     kernel32:KERNEL32.dll
 0001:00000090       __imp__GetOEMCP@0          10001090     kernel32:KERNEL32.dll
 0001:00000094       __imp__IsValidCodePage@4   10001094     kernel32:KERNEL32.dll
 0001:00000098       __imp__TlsAlloc@0          10001098     kernel32:KERNEL32.dll
 0001:0000009c       __imp__TlsGetValue@4       1000109c     kernel32:KERNEL32.dll
 0001:000000a0       __imp__TlsSetValue@8       100010a0     kernel32:KERNEL32.dll
 0001:000000a4       __imp__TlsFree@4           100010a4     kernel32:KERNEL32.dll
 0001:000000a8       __imp__SetLastError@4      100010a8     kernel32:KERNEL32.dll
 0001:000000ac       __imp__Sleep@4             100010ac     kernel32:KERNEL32.dll
 0001:000000b0       __imp__SetHandleCount@4    100010b0     kernel32:KERNEL32.dll
 0001:000000b4       __imp__InitializeCriticalSectionAndSpinCount@8 100010b4     kernel32:KERNEL32.dll
 0001:000000b8       __imp__GetFileType@4       100010b8     kernel32:KERNEL32.dll
 0001:000000bc       __imp__GetStartupInfoW@4   100010bc     kernel32:KERNEL32.dll
 0001:000000c0       __imp__DeleteCriticalSection@4 100010c0     kernel32:KERNEL32.dll
 0001:000000c4       __imp__GetModuleFileNameA@12 100010c4     kernel32:KERNEL32.dll
 0001:000000c8       __imp__FreeEnvironmentStringsW@4 100010c8     kernel32:KERNEL32.dll
 0001:000000cc       __imp__WideCharToMultiByte@32 100010cc     kernel32:KERNEL32.dll
 0001:000000d0       __imp__GetEnvironmentStringsW@0 100010d0     kernel32:KERNEL32.dll
 0001:000000d4       __imp__QueryPerformanceCounter@4 100010d4     kernel32:KERNEL32.dll
 0001:000000d8       __imp__GetCurrentProcessId@0 100010d8     kernel32:KERNEL32.dll
 0001:000000dc       __imp__GetSystemTimeAsFileTime@4 100010dc     kernel32:KERNEL32.dll
 0001:000000e0       __imp__RaiseException@16   100010e0     kernel32:KERNEL32.dll
 0001:000000e4       __imp__UnhandledExceptionFilter@4 100010e4     kernel32:KERNEL32.dll
 0001:000000e8       __imp__SetUnhandledExceptionFilter@4 100010e8     kernel32:KERNEL32.dll
 0001:000000ec       __imp__IsDebuggerPresent@0 100010ec     kernel32:KERNEL32.dll
 0001:000000f0       __imp__TerminateProcess@8  100010f0     kernel32:KERNEL32.dll
 0001:000000f4       __imp__GetCurrentProcess@0 100010f4     kernel32:KERNEL32.dll
 0001:000000f8       __imp__LeaveCriticalSection@4 100010f8     kernel32:KERNEL32.dll
 0001:000000fc       __imp__EnterCriticalSection@4 100010fc     kernel32:KERNEL32.dll
 0001:00000100       __imp__LoadLibraryW@4      10001100     kernel32:KERNEL32.dll
 0001:00000104       __imp__LCMapStringW@24     10001104     kernel32:KERNEL32.dll
 0001:00000108       __imp__MultiByteToWideChar@24 10001108     kernel32:KERNEL32.dll
 0001:0000010c       __imp__GetStringTypeW@16   1000110c     kernel32:KERNEL32.dll
 0001:00000110       __imp__RtlUnwind@16        10001110     kernel32:KERNEL32.dll
 0001:00000114       __imp__HeapSize@12         10001114     kernel32:KERNEL32.dll
 0001:00000118       \177KERNEL32_NULL_THUNK_DATA 10001118     kernel32:KERNEL32.dll
 0001:0000011c       ___xc_a                    1000111c     LIBCMT:crt0init.obj
 0001:00000120       ___xc_z                    10001120     LIBCMT:crt0init.obj
 0001:00000124       ___xi_a                    10001124     LIBCMT:crt0init.obj
 0001:00000134       ___xi_z                    10001134     LIBCMT:crt0init.obj
 0001:00000138       ___xp_a                    10001138     LIBCMT:crt0init.obj
 0001:0000013c       ___xp_z                    1000113c     LIBCMT:crt0init.obj
 0001:00000140       ___xt_a                    10001140     LIBCMT:crt0init.obj
 0001:00000144       ___xt_z                    10001144     LIBCMT:crt0init.obj
 0001:00000158       _MainGuid                  10001158     Compare.obj
 0001:00000168       _MenuGuid                  10001168     Compare.obj
 0001:00000178       _DialogGuid                10001178     Compare.obj
 0001:00000188       ??_C@_1BG@EEJFCAOO@?$AAS?$AAh?$AAo?$AAw?$AAH?$AAi?$AAd?$AAd?$AAe?$AAn?$AA?$AA@ 10001188     Compare.obj
 0001:000001a0       ??_C@_1BC@ENICKDH@?$AAC?$AAo?$AAn?$AAt?$AAe?$AAn?$AAt?$AAs?$AA?$AA@ 100011a0     Compare.obj
 0001:000001b4       ??_C@_11LOCGONAA@?$AA?$AA@ 100011b4     Compare.obj
 0001:000001b8       ??_C@_1M@KNJIDFOP@?$AA9?$AA9?$AA9?$AA9?$AA9?$AA?$AA@ 100011b8     Compare.obj
 0001:000001c4       ??_C@_1CE@FBOAEKEI@?$AAP?$AAr?$AAo?$AAc?$AAe?$AAs?$AAs?$AAS?$AAu?$AAb?$AAf?$AAo?$AAl?$AAd?$AAe?$AAr?$AAs?$AA?$AA@ 100011c4     Compare.obj
 0001:000001e8       ??_C@_1CA@KJDAALFO@?$AAU?$AAs?$AAe?$AAM?$AAa?$AAx?$AAS?$AAc?$AAa?$AAn?$AAD?$AAe?$AAp?$AAt?$AAh?$AA?$AA@ 100011e8     Compare.obj
 0001:00000208       ??_C@_1BK@GGEMFANC@?$AAM?$AAa?$AAx?$AAS?$AAc?$AAa?$AAn?$AAD?$AAe?$AAp?$AAt?$AAh?$AA?$AA@ 10001208     Compare.obj
 0001:00000224       ??_C@_1CA@MDABALAC@?$AAP?$AAr?$AAo?$AAc?$AAe?$AAs?$AAs?$AAS?$AAe?$AAl?$AAe?$AAc?$AAt?$AAe?$AAd?$AA?$AA@ 10001224     Compare.obj
 0001:00000244       ??_C@_1BI@HJKFLAP@?$AAC?$AAo?$AAm?$AAp?$AAa?$AAr?$AAe?$AAT?$AAi?$AAm?$AAe?$AA?$AA@ 10001244     Compare.obj
 0001:0000025c       ??_C@_1CC@GIIFACBC@?$AAL?$AAo?$AAw?$AAP?$AAr?$AAe?$AAc?$AAi?$AAs?$AAi?$AAo?$AAn?$AAT?$AAi?$AAm?$AAe?$AA?$AA@ 1000125c     Compare.obj
 0001:00000280       ??_C@_1EE@EFHMKIOD@?$AAI?$AAg?$AAn?$AAo?$AAr?$AAe?$AAP?$AAo?$AAs?$AAs?$AAi?$AAb?$AAl?$AAe?$AAT?$AAi?$AAm?$AAe?$AAZ?$AAo?$AAn?$AAe?$AAD?$AAi?$AAf?$AAf?$AAe?$AAr?$AAe?$AAn?$AAc?$AAe@ 10001280     Compare.obj
 0001:000002c4       ??_C@_1BI@PLJFHCFF@?$AAC?$AAo?$AAm?$AAp?$AAa?$AAr?$AAe?$AAS?$AAi?$AAz?$AAe?$AA?$AA@ 100012c4     Compare.obj
 0001:000002dc       ??_C@_1CA@JKHJMABM@?$AAC?$AAo?$AAm?$AAp?$AAa?$AAr?$AAe?$AAC?$AAo?$AAn?$AAt?$AAe?$AAn?$AAt?$AAs?$AA?$AA@ 100012dc     Compare.obj
 0001:000002fc       ??_C@_1CM@MCIOEKOG@?$AAC?$AAo?$AAm?$AAp?$AAa?$AAr?$AAe?$AAC?$AAo?$AAn?$AAt?$AAe?$AAn?$AAt?$AAs?$AAI?$AAg?$AAn?$AAo?$AAr?$AAe?$AA?$AA@ 100012fc     Compare.obj
 0001:00000328       ??_C@_1BO@PEKJDKMD@?$AAI?$AAg?$AAn?$AAo?$AAr?$AAe?$AAN?$AAe?$AAw?$AAL?$AAi?$AAn?$AAe?$AAs?$AA?$AA@ 10001328     Compare.obj
 0001:00000348       ??_C@_1CC@EJJKPBBK@?$AAI?$AAg?$AAn?$AAo?$AAr?$AAe?$AAW?$AAh?$AAi?$AAt?$AAe?$AAs?$AAp?$AAa?$AAc?$AAe?$AA?$AA@ 10001348     Compare.obj
 0001:0000036c       ??_C@_1CE@FJPIMCHB@?$AAM?$AAe?$AAs?$AAs?$AAa?$AAg?$AAe?$AAW?$AAh?$AAe?$AAn?$AAN?$AAo?$AAD?$AAi?$AAf?$AAf?$AA?$AA@ 1000136c     Compare.obj
 0001:00000390       ??_C@_17FPIFMLJN@?$AAE?$AAs?$AAc?$AA?$AA@ 10001390     Compare.obj
 0001:00000398       ??_C@_19MJCDBCKE@?$AA?2?$AA?2?$AA?$DP?$AA?2?$AA?$AA@ 10001398     Compare.obj
 0001:000003a4       ??_C@_13JOFGPIOO@?$AA?4?$AA?$AA@ 100013a4     Compare.obj
 0001:000003a8       ??_C@_15DDHGOCBH@?$AA?4?$AA?4?$AA?$AA@ 100013a8     Compare.obj
 0001:000003b0       ??_C@_1DE@BGKMIKPD@?$AAE?$AAu?$AAg?$AAe?$AAn?$AAe?$AA?5?$AAR?$AAo?$AAs?$AAh?$AAa?$AAl?$AA?5?$AA?$CG?$AA?5?$AAF?$AAa?$AAr?$AA?5?$AAG?$AAr?$AAo?$AAu?$AAp?$AA?$AA@ 100013b0     Compare.obj
 0001:000003e8       ??_C@_1EM@KDLPMJGE@?$AAA?$AAd?$AAv?$AAa?$AAn?$AAc?$AAe?$AAd?$AA?5?$AAF?$AAi?$AAl?$AAe?$AA?5?$AAC?$AAo?$AAm?$AAp?$AAa?$AAr?$AAe?$AA?5?$AAf?$AAo?$AAr?$AA?5?$AAF?$AAa?$AAr?$AA?5?$AAM?$AAa@ 100013e8     Compare.obj
 0001:00000434       ??_C@_1BA@NIFMCONN@?$AAC?$AAo?$AAm?$AAp?$AAa?$AAr?$AAe?$AA?$AA@ 10001434     Compare.obj
 0001:00000444       ??_C@_17LGKOMLJ@?$AA?4?$AA?4?$AA?4?$AA?$AA@ 10001444     Compare.obj
 0001:0000044c       ??_C@_15PKPONJIK@?$AA?2?$AA?$CK?$AA?$AA@ 1000144c     Compare.obj
 0001:00000454       ??_C@_13BBDEGPLJ@?$AA?$CK?$AA?$AA@ 10001454     Compare.obj
 0001:00000458       ??_C@_1CE@FMMDKAAJ@?$AAC?$AAo?$AAm?$AAp?$AAa?$AAr?$AAe?$AAB?$AAu?$AAf?$AAf?$AAe?$AAr?$AAS?$AAi?$AAz?$AAe?$AA?$AA@ 10001458     Compare.obj
 0001:0000047c       ??_C@_1O@PNMIMBDD@?$AAC?$AAO?$AAN?$AAI?$AAN?$AA$?$AA?$AA@ 1000147c     Compare.obj
 0001:0000048c       __pDefaultRawDllMain       1000148c     LIBCMT:dllcrt0.obj
 0001:0000048c       __pRawDllMain              1000148c     LIBCMT:dllcrt0.obj
 0001:00000494       ??_7bad_alloc@std@@6B@     10001494     LIBCMT:new.obj
 0001:0000049c       ??_C@_0P@GHFPNOJB@bad?5allocation?$AA@ 1000149c     LIBCMT:new.obj
 0001:000004ac       ??_C@_0P@MIGLKIOC@CorExitProcess?$AA@ 100014ac     LIBCMT:crt0dat.obj
 0001:000004bc       ??_C@_1BI@BGOHAHKC@?$AAm?$AAs?$AAc?$AAo?$AAr?$AAe?$AAe?$AA?4?$AAd?$AAl?$AAl?$AA?$AA@ 100014bc     LIBCMT:crt0dat.obj
 0001:000004d4       ??_C@_1BO@BKOMIGKJ@?$AAr?$AAu?$AAn?$AAt?$AAi?$AAm?$AAe?$AA?5?$AAe?$AAr?$AAr?$AAo?$AAr?$AA?5?$AA?$AA@ 100014d4     LIBCMT:crt0msg.obj
 0001:000004f4       ??_C@_15JNBOKNOG@?$AA?$AN?$AA?6?$AA?$AA@ 100014f4     LIBCMT:crt0msg.obj
 0001:000004fc       ??_C@_1BM@JBBEPPHI@?$AAT?$AAL?$AAO?$AAS?$AAS?$AA?5?$AAe?$AAr?$AAr?$AAo?$AAr?$AA?$AN?$AA?6?$AA?$AA@ 100014fc     LIBCMT:crt0msg.obj
 0001:00000518       ??_C@_1BK@KMOMNAAI@?$AAS?$AAI?$AAN?$AAG?$AA?5?$AAe?$AAr?$AAr?$AAo?$AAr?$AA?$AN?$AA?6?$AA?$AA@ 10001518     LIBCMT:crt0msg.obj
 0001:00000534       ??_C@_1BO@BFCDCGC@?$AAD?$AAO?$AAM?$AAA?$AAI?$AAN?$AA?5?$AAe?$AAr?$AAr?$AAo?$AAr?$AA?$AN?$AA?6?$AA?$AA@ 10001534     LIBCMT:crt0msg.obj
 0001:00000558       ??_C@_1BOO@KGEDBGAJ@?$AAR?$AA6?$AA0?$AA3?$AA3?$AA?$AN?$AA?6?$AA?9?$AA?5?$AAA?$AAt?$AAt?$AAe?$AAm?$AAp?$AAt?$AA?5?$AAt?$AAo?$AA?5?$AAu?$AAs?$AAe?$AA?5?$AAM?$AAS?$AAI?$AAL?$AA?5?$AAc?$AAo?$AAd@ 10001558     LIBCMT:crt0msg.obj
 0001:00000748       ??_C@_1GG@GOPILAJP@?$AAR?$AA6?$AA0?$AA3?$AA2?$AA?$AN?$AA?6?$AA?9?$AA?5?$AAn?$AAo?$AAt?$AA?5?$AAe?$AAn?$AAo?$AAu?$AAg?$AAh?$AA?5?$AAs?$AAp?$AAa?$AAc?$AAe?$AA?5?$AAf?$AAo?$AAr?$AA?5?$AAl?$AAo@ 10001748     LIBCMT:crt0msg.obj
 0001:000007b0       ??_C@_1MG@ENCOOIDF@?$AAR?$AA6?$AA0?$AA3?$AA1?$AA?$AN?$AA?6?$AA?9?$AA?5?$AAA?$AAt?$AAt?$AAe?$AAm?$AAp?$AAt?$AA?5?$AAt?$AAo?$AA?5?$AAi?$AAn?$AAi?$AAt?$AAi?$AAa?$AAl?$AAi?$AAz?$AAe?$AA?5?$AAt@ 100017b0     LIBCMT:crt0msg.obj
 0001:00000878       ??_C@_1DO@BMFCDCD@?$AAR?$AA6?$AA0?$AA3?$AA0?$AA?$AN?$AA?6?$AA?9?$AA?5?$AAC?$AAR?$AAT?$AA?5?$AAn?$AAo?$AAt?$AA?5?$AAi?$AAn?$AAi?$AAt?$AAi?$AAa?$AAl?$AAi?$AAz?$AAe?$AAd?$AA?$AN?$AA?6?$AA?$AA@ 10001878     LIBCMT:crt0msg.obj
 0001:000008b8       ??_C@_1EK@HHFLMAOL@?$AAR?$AA6?$AA0?$AA2?$AA8?$AA?$AN?$AA?6?$AA?9?$AA?5?$AAu?$AAn?$AAa?$AAb?$AAl?$AAe?$AA?5?$AAt?$AAo?$AA?5?$AAi?$AAn?$AAi?$AAt?$AAi?$AAa?$AAl?$AAi?$AAz?$AAe?$AA?5?$AAh?$AAe@ 100018b8     LIBCMT:crt0msg.obj
 0001:00000908       ??_C@_1GK@MFGOKLAG@?$AAR?$AA6?$AA0?$AA2?$AA7?$AA?$AN?$AA?6?$AA?9?$AA?5?$AAn?$AAo?$AAt?$AA?5?$AAe?$AAn?$AAo?$AAu?$AAg?$AAh?$AA?5?$AAs?$AAp?$AAa?$AAc?$AAe?$AA?5?$AAf?$AAo?$AAr?$AA?5?$AAl?$AAo@ 10001908     LIBCMT:crt0msg.obj
 0001:00000978       ??_C@_1GK@MCAAGJMO@?$AAR?$AA6?$AA0?$AA2?$AA6?$AA?$AN?$AA?6?$AA?9?$AA?5?$AAn?$AAo?$AAt?$AA?5?$AAe?$AAn?$AAo?$AAu?$AAg?$AAh?$AA?5?$AAs?$AAp?$AAa?$AAc?$AAe?$AA?5?$AAf?$AAo?$AAr?$AA?5?$AAs?$AAt@ 10001978     LIBCMT:crt0msg.obj
 0001:000009e8       ??_C@_1EM@MAADIHMB@?$AAR?$AA6?$AA0?$AA2?$AA5?$AA?$AN?$AA?6?$AA?9?$AA?5?$AAp?$AAu?$AAr?$AAe?$AA?5?$AAv?$AAi?$AAr?$AAt?$AAu?$AAa?$AAl?$AA?5?$AAf?$AAu?$AAn?$AAc?$AAt?$AAi?$AAo?$AAn?$AA?5?$AAc@ 100019e8     LIBCMT:crt0msg.obj
 0001:00000a38       ??_C@_1GK@FHCKBEFA@?$AAR?$AA6?$AA0?$AA2?$AA4?$AA?$AN?$AA?6?$AA?9?$AA?5?$AAn?$AAo?$AAt?$AA?5?$AAe?$AAn?$AAo?$AAu?$AAg?$AAh?$AA?5?$AAs?$AAp?$AAa?$AAc?$AAe?$AA?5?$AAf?$AAo?$AAr?$AA?5?$AA_?$AAo@ 10001a38     LIBCMT:crt0msg.obj
 0001:00000aa8       ??_C@_1FC@ECHBIFBC@?$AAR?$AA6?$AA0?$AA1?$AA9?$AA?$AN?$AA?6?$AA?9?$AA?5?$AAu?$AAn?$AAa?$AAb?$AAl?$AAe?$AA?5?$AAt?$AAo?$AA?5?$AAo?$AAp?$AAe?$AAn?$AA?5?$AAc?$AAo?$AAn?$AAs?$AAo?$AAl?$AAe?$AA?5@ 10001aa8     LIBCMT:crt0msg.obj
 0001:00000b00       ??_C@_1EC@JIBHAOPH@?$AAR?$AA6?$AA0?$AA1?$AA8?$AA?$AN?$AA?6?$AA?9?$AA?5?$AAu?$AAn?$AAe?$AAx?$AAp?$AAe?$AAc?$AAt?$AAe?$AAd?$AA?5?$AAh?$AAe?$AAa?$AAp?$AA?5?$AAe?$AAr?$AAr?$AAo?$AAr?$AA?$AN?$AA?6@ 10001b00     LIBCMT:crt0msg.obj
 0001:00000b48       ??_C@_1FK@BEOGODMC@?$AAR?$AA6?$AA0?$AA1?$AA7?$AA?$AN?$AA?6?$AA?9?$AA?5?$AAu?$AAn?$AAe?$AAx?$AAp?$AAe?$AAc?$AAt?$AAe?$AAd?$AA?5?$AAm?$AAu?$AAl?$AAt?$AAi?$AAt?$AAh?$AAr?$AAe?$AAa?$AAd?$AA?5@ 10001b48     LIBCMT:crt0msg.obj
 0001:00000ba8       ??_C@_1FI@LOGNIKDM@?$AAR?$AA6?$AA0?$AA1?$AA6?$AA?$AN?$AA?6?$AA?9?$AA?5?$AAn?$AAo?$AAt?$AA?5?$AAe?$AAn?$AAo?$AAu?$AAg?$AAh?$AA?5?$AAs?$AAp?$AAa?$AAc?$AAe?$AA?5?$AAf?$AAo?$AAr?$AA?5?$AAt?$AAh@ 10001ba8     LIBCMT:crt0msg.obj
 0001:00000c00       ??_C@_1EG@BEHAGFJD@?$AAR?$AA6?$AA0?$AA1?$AA0?$AA?$AN?$AA?6?$AA?9?$AA?5?$AAa?$AAb?$AAo?$AAr?$AAt?$AA?$CI?$AA?$CJ?$AA?5?$AAh?$AAa?$AAs?$AA?5?$AAb?$AAe?$AAe?$AAn?$AA?5?$AAc?$AAa?$AAl?$AAl?$AAe?$AAd@ 10001c00     LIBCMT:crt0msg.obj
 0001:00000c48       ??_C@_1FI@HONFMGBI@?$AAR?$AA6?$AA0?$AA0?$AA9?$AA?$AN?$AA?6?$AA?9?$AA?5?$AAn?$AAo?$AAt?$AA?5?$AAe?$AAn?$AAo?$AAu?$AAg?$AAh?$AA?5?$AAs?$AAp?$AAa?$AAc?$AAe?$AA?5?$AAf?$AAo?$AAr?$AA?5?$AAe?$AAn@ 10001c48     LIBCMT:crt0msg.obj
 0001:00000ca0       ??_C@_1FE@LLNEDJMD@?$AAR?$AA6?$AA0?$AA0?$AA8?$AA?$AN?$AA?6?$AA?9?$AA?5?$AAn?$AAo?$AAt?$AA?5?$AAe?$AAn?$AAo?$AAu?$AAg?$AAh?$AA?5?$AAs?$AAp?$AAa?$AAc?$AAe?$AA?5?$AAf?$AAo?$AAr?$AA?5?$AAa?$AAr@ 10001ca0     LIBCMT:crt0msg.obj
 0001:00000cf8       ??_C@_1FK@PGACCAFB@?$AAR?$AA6?$AA0?$AA0?$AA2?$AA?$AN?$AA?6?$AA?9?$AA?5?$AAf?$AAl?$AAo?$AAa?$AAt?$AAi?$AAn?$AAg?$AA?5?$AAp?$AAo?$AAi?$AAn?$AAt?$AA?5?$AAs?$AAu?$AAp?$AAp?$AAo?$AAr?$AAt?$AA?5@ 10001cf8     LIBCMT:crt0msg.obj
 0001:00000e08       ??_C@_1EK@MBDPDCGA@?$AAM?$AAi?$AAc?$AAr?$AAo?$AAs?$AAo?$AAf?$AAt?$AA?5?$AAV?$AAi?$AAs?$AAu?$AAa?$AAl?$AA?5?$AAC?$AA?$CL?$AA?$CL?$AA?5?$AAR?$AAu?$AAn?$AAt?$AAi?$AAm?$AAe?$AA?5?$AAL?$AAi?$AAb@ 10001e08     LIBCMT:crt0msg.obj
 0001:00000e54       ??_C@_15IABLJNFO@?$AA?6?$AA?6?$AA?$AA@ 10001e54     LIBCMT:crt0msg.obj
 0001:00000e5c       ??_C@_1CO@EAEJAADC@?$AA?$DM?$AAp?$AAr?$AAo?$AAg?$AAr?$AAa?$AAm?$AA?5?$AAn?$AAa?$AAm?$AAe?$AA?5?$AAu?$AAn?$AAk?$AAn?$AAo?$AAw?$AAn?$AA?$DO?$AA?$AA@ 10001e5c     LIBCMT:crt0msg.obj
 0001:00000e8c       ??_C@_1DE@JNGNBFGO@?$AAR?$AAu?$AAn?$AAt?$AAi?$AAm?$AAe?$AA?5?$AAE?$AAr?$AAr?$AAo?$AAr?$AA?$CB?$AA?6?$AA?6?$AAP?$AAr?$AAo?$AAg?$AAr?$AAa?$AAm?$AA?3?$AA?5?$AA?$AA@ 10001e8c     LIBCMT:crt0msg.obj
 0001:00000ec0       ??_C@_1BC@GDGBMEMK@?$AAH?$AAH?$AA?3?$AAm?$AAm?$AA?3?$AAs?$AAs?$AA?$AA@ 10001ec0     LIBCMT:nlsdata2.obj
 0001:00000ed4       ??_C@_1CI@KNAKOEBC@?$AAd?$AAd?$AAd?$AAd?$AA?0?$AA?5?$AAM?$AAM?$AAM?$AAM?$AA?5?$AAd?$AAd?$AA?0?$AA?5?$AAy?$AAy?$AAy?$AAy?$AA?$AA@ 10001ed4     LIBCMT:nlsdata2.obj
 0001:00000efc       ??_C@_1BC@IEBCMHCM@?$AAM?$AAM?$AA?1?$AAd?$AAd?$AA?1?$AAy?$AAy?$AA?$AA@ 10001efc     LIBCMT:nlsdata2.obj
 0001:00000f10       ??_C@_15CLMNNGEL@?$AAP?$AAM?$AA?$AA@ 10001f10     LIBCMT:nlsdata2.obj
 0001:00000f18       ??_C@_15ODEHAHHF@?$AAA?$AAM?$AA?$AA@ 10001f18     LIBCMT:nlsdata2.obj
 0001:00000f20       ??_C@_1BC@FEMKIFH@?$AAD?$AAe?$AAc?$AAe?$AAm?$AAb?$AAe?$AAr?$AA?$AA@ 10001f20     LIBCMT:nlsdata2.obj
 0001:00000f34       ??_C@_1BC@BGLIFPF@?$AAN?$AAo?$AAv?$AAe?$AAm?$AAb?$AAe?$AAr?$AA?$AA@ 10001f34     LIBCMT:nlsdata2.obj
 0001:00000f48       ??_C@_1BA@EPANDLNG@?$AAO?$AAc?$AAt?$AAo?$AAb?$AAe?$AAr?$AA?$AA@ 10001f48     LIBCMT:nlsdata2.obj
 0001:00000f58       ??_C@_1BE@DKAAMBJL@?$AAS?$AAe?$AAp?$AAt?$AAe?$AAm?$AAb?$AAe?$AAr?$AA?$AA@ 10001f58     LIBCMT:nlsdata2.obj
 0001:00000f6c       ??_C@_1O@PAHLKOAC@?$AAA?$AAu?$AAg?$AAu?$AAs?$AAt?$AA?$AA@ 10001f6c     LIBCMT:nlsdata2.obj
 0001:00000f7c       ??_C@_19BIFMLPCD@?$AAJ?$AAu?$AAl?$AAy?$AA?$AA@ 10001f7c     LIBCMT:nlsdata2.obj
 0001:00000f88       ??_C@_19EPFLPGAP@?$AAJ?$AAu?$AAn?$AAe?$AA?$AA@ 10001f88     LIBCMT:nlsdata2.obj
 0001:00000f94       ??_C@_1M@GJNLMHFD@?$AAA?$AAp?$AAr?$AAi?$AAl?$AA?$AA@ 10001f94     LIBCMT:nlsdata2.obj
 0001:00000fa0       ??_C@_1M@IKEENEDF@?$AAM?$AAa?$AAr?$AAc?$AAh?$AA?$AA@ 10001fa0     LIBCMT:nlsdata2.obj
 0001:00000fac       ??_C@_1BC@JGDDFFAM@?$AAF?$AAe?$AAb?$AAr?$AAu?$AAa?$AAr?$AAy?$AA?$AA@ 10001fac     LIBCMT:nlsdata2.obj
 0001:00000fc0       ??_C@_1BA@EFMEIEBA@?$AAJ?$AAa?$AAn?$AAu?$AAa?$AAr?$AAy?$AA?$AA@ 10001fc0     LIBCMT:nlsdata2.obj
 0001:00000fd0       ??_C@_17EGKACKIF@?$AAD?$AAe?$AAc?$AA?$AA@ 10001fd0     LIBCMT:nlsdata2.obj
 0001:00000fd8       ??_C@_17BBDMLCIG@?$AAN?$AAo?$AAv?$AA?$AA@ 10001fd8     LIBCMT:nlsdata2.obj
 0001:00000fe0       ??_C@_17FNLKOI@?$AAO?$AAc?$AAt?$AA?$AA@ 10001fe0     LIBCMT:nlsdata2.obj
 0001:00000fe8       ??_C@_17HCHCOKMG@?$AAS?$AAe?$AAp?$AA?$AA@ 10001fe8     LIBCMT:nlsdata2.obj
 0001:00000ff0       ??_C@_17ICPELBCN@?$AAA?$AAu?$AAg?$AA?$AA@ 10001ff0     LIBCMT:nlsdata2.obj
 0001:00000ff8       ??_C@_17IJPCKHK@?$AAJ?$AAu?$AAl?$AA?$AA@ 10001ff8     LIBCMT:nlsdata2.obj
 0001:00001000       ??_C@_17KCJGOCPB@?$AAJ?$AAu?$AAn?$AA?$AA@ 10002000     LIBCMT:nlsdata2.obj
 0001:00001008       ??_C@_17PNNKMEED@?$AAM?$AAa?$AAy?$AA?$AA@ 10002008     LIBCMT:nlsdata2.obj
 0001:00001010       ??_C@_17LFPOIHDD@?$AAA?$AAp?$AAr?$AA?$AA@ 10002010     LIBCMT:nlsdata2.obj
 0001:00001018       ??_C@_17CKNLEDEC@?$AAM?$AAa?$AAr?$AA?$AA@ 10002018     LIBCMT:nlsdata2.obj
 0001:00001020       ??_C@_17LMDJEKJN@?$AAF?$AAe?$AAb?$AA?$AA@ 10002020     LIBCMT:nlsdata2.obj
 0001:00001028       ??_C@_17DKNBKCHM@?$AAJ?$AAa?$AAn?$AA?$AA@ 10002028     LIBCMT:nlsdata2.obj
 0001:00001030       ??_C@_1BC@ENMNNPAJ@?$AAS?$AAa?$AAt?$AAu?$AAr?$AAd?$AAa?$AAy?$AA?$AA@ 10002030     LIBCMT:nlsdata2.obj
 0001:00001044       ??_C@_1O@PDICJHAG@?$AAF?$AAr?$AAi?$AAd?$AAa?$AAy?$AA?$AA@ 10002044     LIBCMT:nlsdata2.obj
 0001:00001054       ??_C@_1BC@HHMNLIHE@?$AAT?$AAh?$AAu?$AAr?$AAs?$AAd?$AAa?$AAy?$AA?$AA@ 10002054     LIBCMT:nlsdata2.obj
 0001:00001068       ??_C@_1BE@EBOGMDOH@?$AAW?$AAe?$AAd?$AAn?$AAe?$AAs?$AAd?$AAa?$AAy?$AA?$AA@ 10002068     LIBCMT:nlsdata2.obj
 0001:0000107c       ??_C@_1BA@ENFBFFEK@?$AAT?$AAu?$AAe?$AAs?$AAd?$AAa?$AAy?$AA?$AA@ 1000207c     LIBCMT:nlsdata2.obj
 0001:0000108c       ??_C@_1O@MMNBFLIA@?$AAM?$AAo?$AAn?$AAd?$AAa?$AAy?$AA?$AA@ 1000208c     LIBCMT:nlsdata2.obj
 0001:0000109c       ??_C@_1O@IHNHDHPB@?$AAS?$AAu?$AAn?$AAd?$AAa?$AAy?$AA?$AA@ 1000209c     LIBCMT:nlsdata2.obj
 0001:000010ac       ??_C@_17GGIBDPIH@?$AAS?$AAa?$AAt?$AA?$AA@ 100020ac     LIBCMT:nlsdata2.obj
 0001:000010b4       ??_C@_17HFOLPPLP@?$AAF?$AAr?$AAi?$AA?$AA@ 100020b4     LIBCMT:nlsdata2.obj
 0001:000010bc       ??_C@_17PDPHAADD@?$AAT?$AAh?$AAu?$AA?$AA@ 100020bc     LIBCMT:nlsdata2.obj
 0001:000010c4       ??_C@_17CJEDCEPE@?$AAW?$AAe?$AAd?$AA?$AA@ 100020c4     LIBCMT:nlsdata2.obj
 0001:000010cc       ??_C@_17BMKGEGOJ@?$AAT?$AAu?$AAe?$AA?$AA@ 100020cc     LIBCMT:nlsdata2.obj
 0001:000010d4       ??_C@_17KBOMKBF@?$AAM?$AAo?$AAn?$AA?$AA@ 100020d4     LIBCMT:nlsdata2.obj
 0001:000010dc       ??_C@_17MBGCMIPB@?$AAS?$AAu?$AAn?$AA?$AA@ 100020dc     LIBCMT:nlsdata2.obj
 0001:000010e4       ??_C@_08JCCMCCIL@HH?3mm?3ss?$AA@ 100020e4     LIBCMT:nlsdata2.obj
 0001:000010f0       ??_C@_0BE@CKGJFCPC@dddd?0?5MMMM?5dd?0?5yyyy?$AA@ 100020f0     LIBCMT:nlsdata2.obj
 0001:00001104       ??_C@_08BPBNCDIB@MM?1dd?1yy?$AA@ 10002104     LIBCMT:nlsdata2.obj
 0001:00001110       ??_C@_02CJNFDJBF@PM?$AA@   10002110     LIBCMT:nlsdata2.obj
 0001:00001114       ??_C@_02DEDBPAFC@AM?$AA@   10002114     LIBCMT:nlsdata2.obj
 0001:00001118       ??_C@_08EDHMEBNP@December?$AA@ 10002118     LIBCMT:nlsdata2.obj
 0001:00001124       ??_C@_08HCHEGEOA@November?$AA@ 10002124     LIBCMT:nlsdata2.obj
 0001:00001130       ??_C@_07JJNFCEND@October?$AA@ 10002130     LIBCMT:nlsdata2.obj
 0001:00001138       ??_C@_09BHHEALKD@September?$AA@ 10002138     LIBCMT:nlsdata2.obj
 0001:00001144       ??_C@_06LBBHFDDG@August?$AA@ 10002144     LIBCMT:nlsdata2.obj
 0001:0000114c       ??_C@_04MIEPOIFP@July?$AA@ 1000214c     LIBCMT:nlsdata2.obj
 0001:00001154       ??_C@_04CNLMGBGM@June?$AA@ 10002154     LIBCMT:nlsdata2.obj
 0001:0000115c       ??_C@_05DMJDNLEJ@April?$AA@ 1000215c     LIBCMT:nlsdata2.obj
 0001:00001164       ??_C@_05HPCKOFNC@March?$AA@ 10002164     LIBCMT:nlsdata2.obj
 0001:0000116c       ??_C@_08GNJGEPFN@February?$AA@ 1000216c     LIBCMT:nlsdata2.obj
 0001:00001178       ??_C@_07CGJPFGJA@January?$AA@ 10002178     LIBCMT:nlsdata2.obj
 0001:00001180       ??_C@_03MKABNOCG@Dec?$AA@  10002180     LIBCMT:nlsdata2.obj
 0001:00001184       ??_C@_03JPJOFNIA@Nov?$AA@  10002184     LIBCMT:nlsdata2.obj
 0001:00001188       ??_C@_03BMAOKBAD@Oct?$AA@  10002188     LIBCMT:nlsdata2.obj
 0001:0000118c       ??_C@_03GGCAPAJC@Sep?$AA@  1000218c     LIBCMT:nlsdata2.obj
 0001:00001190       ??_C@_03IFJFEIGA@Aug?$AA@  10002190     LIBCMT:nlsdata2.obj
 0001:00001194       ??_C@_03LBGABGKK@Jul?$AA@  10002194     LIBCMT:nlsdata2.obj
 0001:00001198       ??_C@_03IDFGHECI@Jun?$AA@  10002198     LIBCMT:nlsdata2.obj
 0001:0000119c       ??_C@_03CNMDKL@May?$AA@    1000219c     LIBCMT:nlsdata2.obj
 0001:000011a0       ??_C@_03LEOLGMJP@Apr?$AA@  100021a0     LIBCMT:nlsdata2.obj
 0001:000011a4       ??_C@_03ODNJBKGA@Mar?$AA@  100021a4     LIBCMT:nlsdata2.obj
 0001:000011a8       ??_C@_03HJBDCHOM@Feb?$AA@  100021a8     LIBCMT:nlsdata2.obj
 0001:000011ac       ??_C@_03JIHJHPIE@Jan?$AA@  100021ac     LIBCMT:nlsdata2.obj
 0001:000011b0       ??_C@_08INBOOONO@Saturday?$AA@ 100021b0     LIBCMT:nlsdata2.obj
 0001:000011bc       ??_C@_06JECMNKMI@Friday?$AA@ 100021bc     LIBCMT:nlsdata2.obj
 0001:000011c4       ??_C@_08HACCIKIA@Thursday?$AA@ 100021c4     LIBCMT:nlsdata2.obj
 0001:000011d0       ??_C@_09DLIGFAKA@Wednesday?$AA@ 100021d0     LIBCMT:nlsdata2.obj
 0001:000011dc       ??_C@_07BAAGCFCM@Tuesday?$AA@ 100021dc     LIBCMT:nlsdata2.obj
 0001:000011e4       ??_C@_06JLEDEDGH@Monday?$AA@ 100021e4     LIBCMT:nlsdata2.obj
 0001:000011ec       ??_C@_06OOPIFAJ@Sunday?$AA@ 100021ec     LIBCMT:nlsdata2.obj
 0001:000011f4       ??_C@_03FEFJNEK@Sat?$AA@   100021f4     LIBCMT:nlsdata2.obj
 0001:000011f8       ??_C@_03IDIOELNC@Fri?$AA@  100021f8     LIBCMT:nlsdata2.obj
 0001:000011fc       ??_C@_03IOFIKPDN@Thu?$AA@  100021fc     LIBCMT:nlsdata2.obj
 0001:00001200       ??_C@_03MHOMLAJA@Wed?$AA@  10002200     LIBCMT:nlsdata2.obj
 0001:00001204       ??_C@_03NAGEINEP@Tue?$AA@  10002204     LIBCMT:nlsdata2.obj
 0001:00001208       ??_C@_03PDAGKDH@Mon?$AA@   10002208     LIBCMT:nlsdata2.obj
 0001:0000120c       ??_C@_03KOEHGMDN@Sun?$AA@  1000220c     LIBCMT:nlsdata2.obj
 0001:00001210       ??_C@_1BK@DBDEIDLH@?$AAK?$AAE?$AAR?$AAN?$AAE?$AAL?$AA3?$AA2?$AA?4?$AAD?$AAL?$AAL?$AA?$AA@ 10002210     LIBCMT:tidtable.obj
 0001:0000122c       ??_C@_07PEJMOBNF@FlsFree?$AA@ 1000222c     LIBCMT:tidtable.obj
 0001:00001234       ??_C@_0M@JCPCPOEF@FlsSetValue?$AA@ 10002234     LIBCMT:tidtable.obj
 0001:00001240       ??_C@_0M@GDNOONDI@FlsGetValue?$AA@ 10002240     LIBCMT:tidtable.obj
 0001:0000124c       ??_C@_08KNHFBNJ@FlsAlloc?$AA@ 1000224c     LIBCMT:tidtable.obj
 0001:000012d8       ??_C@_01NEMOKFLO@?$DN?$AA@ 100022d8     LIBCMT:setlocal.obj
 0001:000012da       ??_C@_00CNPNBAHC@?$AA@     100022da     LIBCMT:setlocal.obj
 0001:000012e0       __XcptActTab               100022e0     LIBCMT:winxfltr.obj
 0001:00001370       __First_FPE_Indx           10002370     LIBCMT:winxfltr.obj
 0001:00001374       __Num_FPE                  10002374     LIBCMT:winxfltr.obj
 0001:00001378       __XcptActTabSize           10002378     LIBCMT:winxfltr.obj
 0001:0000137c       __XcptActTabCount          1000237c     LIBCMT:winxfltr.obj
 0001:00001384       ??_7exception@std@@6B@     10002384     LIBCMT:stdexcpt.obj
 0001:0000138c       ??_C@_0BC@EOODALEL@Unknown?5exception?$AA@ 1000238c     LIBCMT:stdexcpt.obj
 0001:000013a4       ??_7type_info@@6B@         100023a4     LIBCMT:typinfo.obj
 0001:000013c8       ??_C@_0BI@DFKBFLJE@GetProcessWindowStation?$AA@ 100023c8     LIBCMT:crtmboxw.obj
 0001:000013e0       ??_C@_0BK@DEKFELLI@GetUserObjectInformationW?$AA@ 100023e0     LIBCMT:crtmboxw.obj
 0001:000013fc       ??_C@_0BD@HHGDFDBJ@GetLastActivePopup?$AA@ 100023fc     LIBCMT:crtmboxw.obj
 0001:00001410       ??_C@_0BA@HNOPNCHB@GetActiveWindow?$AA@ 10002410     LIBCMT:crtmboxw.obj
 0001:00001420       ??_C@_0M@DLDCCGNP@MessageBoxW?$AA@ 10002420     LIBCMT:crtmboxw.obj
 0001:0000142c       ??_C@_1BG@GOEBHBDC@?$AAU?$AAS?$AAE?$AAR?$AA3?$AA2?$AA?4?$AAD?$AAL?$AAL?$AA?$AA@ 1000242c     LIBCMT:crtmboxw.obj
 0001:00001448       ___newctype                10002448     LIBCMT:ctype.obj
 0001:00001748       __wctype                   10002748     LIBCMT:ctype.obj
 0001:00001950       ___newclmap                10002950     LIBCMT:ctype.obj
 0001:00001ad0       ___newcumap                10002ad0     LIBCMT:ctype.obj
 0001:00001c58       ??_C@_0BK@CFCOFLF@?5Complete?5Object?5Locator?8?$AA@ 10002c58     LIBCMT:undname.obj
 0001:00001c74       ??_C@_0BN@MECKDCOJ@?5Class?5Hierarchy?5Descriptor?8?$AA@ 10002c74     LIBCMT:undname.obj
 0001:00001c94       ??_C@_0BD@LGICGFMM@?5Base?5Class?5Array?8?$AA@ 10002c94     LIBCMT:undname.obj
 0001:00001ca8       ??_C@_0BM@LDKODKLH@?5Base?5Class?5Descriptor?5at?5?$CI?$AA@ 10002ca8     LIBCMT:undname.obj
 0001:00001cc4       ??_C@_0BC@DAFEJGAK@?5Type?5Descriptor?8?$AA@ 10002cc4     LIBCMT:undname.obj
 0001:00001cd8       ??_C@_0BM@PMGGMLDN@?$GAlocal?5static?5thread?5guard?8?$AA@ 10002cd8     LIBCMT:undname.obj
 0001:00001cf4       ??_C@_0CL@FGIJHLCE@?$GAmanaged?5vector?5copy?5constructor@ 10002cf4     LIBCMT:undname.obj
 0001:00001d20       ??_C@_0CJ@GJELGAMM@?$GAvector?5vbase?5copy?5constructor?5i@ 10002d20     LIBCMT:undname.obj
 0001:00001d4c       ??_C@_0CD@CGAJBKEJ@?$GAvector?5copy?5constructor?5iterato@ 10002d4c     LIBCMT:undname.obj
 0001:00001d70       ??_C@_0CB@PDBIFEP@?$GAdynamic?5atexit?5destructor?5for?5?8@ 10002d70     LIBCMT:undname.obj
 0001:00001d94       ??_C@_0BL@CLIPGLGB@?$GAdynamic?5initializer?5for?5?8?$AA@ 10002d94     LIBCMT:undname.obj
 0001:00001db0       ??_C@_0CM@FCBBDIGB@?$GAeh?5vector?5vbase?5copy?5constructo@ 10002db0     LIBCMT:undname.obj
 0001:00001ddc       ??_C@_0CG@HLDDJMAG@?$GAeh?5vector?5copy?5constructor?5iter@ 10002ddc     LIBCMT:undname.obj
 0001:00001e04       ??_C@_0CF@IMGKMJNO@?$GAmanaged?5vector?5destructor?5itera@ 10002e04     LIBCMT:undname.obj
 0001:00001e2c       ??_C@_0CG@CFDHKGGD@?$GAmanaged?5vector?5constructor?5iter@ 10002e2c     LIBCMT:undname.obj
 0001:00001e54       ??_C@_0BN@CKNJLHMB@?$GAplacement?5delete?$FL?$FN?5closure?8?$AA@ 10002e54     LIBCMT:undname.obj
 0001:00001e74       ??_C@_0BL@CNOONJFP@?$GAplacement?5delete?5closure?8?$AA@ 10002e74     LIBCMT:undname.obj
 0001:00001e90       ??_C@_0P@HJKNJFNN@?$GAomni?5callsig?8?$AA@ 10002e90     LIBCMT:undname.obj
 0001:00001ea0       ??_C@_09LBNFPBCA@?5delete?$FL?$FN?$AA@ 10002ea0     LIBCMT:undname.obj
 0001:00001eac       ??_C@_06FHBGPFGH@?5new?$FL?$FN?$AA@ 10002eac     LIBCMT:undname.obj
 0001:00001eb4       ??_C@_0CE@IIHCMGGL@?$GAlocal?5vftable?5constructor?5closu@ 10002eb4     LIBCMT:undname.obj
 0001:00001ed8       ??_C@_0BA@KKLDJDLB@?$GAlocal?5vftable?8?$AA@ 10002ed8     LIBCMT:undname.obj
 0001:00001ee8       ??_C@_05KHLCHHI@?$GARTTI?$AA@ 10002ee8     LIBCMT:undname.obj
 0001:00001ef0       ??_C@_03KLGMFNMG@?$GAEH?$AA@ 10002ef0     LIBCMT:undname.obj
 0001:00001ef4       ??_C@_0BA@KBCDOMBN@?$GAudt?5returning?8?$AA@ 10002ef4     LIBCMT:undname.obj
 0001:00001f04       ??_C@_0BL@LLKPOHJI@?$GAcopy?5constructor?5closure?8?$AA@ 10002f04     LIBCMT:undname.obj
 0001:00001f20       ??_C@_0CH@OOJPLCPH@?$GAeh?5vector?5vbase?5constructor?5ite@ 10002f20     LIBCMT:undname.obj
 0001:00001f48       ??_C@_0CA@GCEOPDGL@?$GAeh?5vector?5destructor?5iterator?8?$AA@ 10002f48     LIBCMT:undname.obj
 0001:00001f68       ??_C@_0CB@JONCMFFK@?$GAeh?5vector?5constructor?5iterator?8@ 10002f68     LIBCMT:undname.obj
 0001:00001f8c       ??_C@_0BL@NILFHHPC@?$GAvirtual?5displacement?5map?8?$AA@ 10002f8c     LIBCMT:undname.obj
 0001:00001fa8       ??_C@_0CE@IKBNEHA@?$GAvector?5vbase?5constructor?5iterat@ 10002fa8     LIBCMT:undname.obj
 0001:00001fcc       ??_C@_0BN@LFPFMEDL@?$GAvector?5destructor?5iterator?8?$AA@ 10002fcc     LIBCMT:undname.obj
 0001:00001fec       ??_C@_0BO@PFGOCPJJ@?$GAvector?5constructor?5iterator?8?$AA@ 10002fec     LIBCMT:undname.obj
 0001:0000200c       ??_C@_0BN@IMDCHIKM@?$GAscalar?5deleting?5destructor?8?$AA@ 1000300c     LIBCMT:undname.obj
 0001:0000202c       ??_C@_0BO@OBMKPJIG@?$GAdefault?5constructor?5closure?8?$AA@ 1000302c     LIBCMT:undname.obj
 0001:0000204c       ??_C@_0BN@DEGPLNFK@?$GAvector?5deleting?5destructor?8?$AA@ 1000304c     LIBCMT:undname.obj
 0001:0000206c       ??_C@_0BD@JDLKDPAB@?$GAvbase?5destructor?8?$AA@ 1000306c     LIBCMT:undname.obj
 0001:00002080       ??_C@_08OBABFOLI@?$GAstring?8?$AA@ 10003080     LIBCMT:undname.obj
 0001:0000208c       ??_C@_0BF@KDPPACIK@?$GAlocal?5static?5guard?8?$AA@ 1000308c     LIBCMT:undname.obj
 0001:000020a4       ??_C@_08LLFFHHDJ@?$GAtypeof?8?$AA@ 100030a4     LIBCMT:undname.obj
 0001:000020b0       ??_C@_07FEEIOKP@?$GAvcall?8?$AA@ 100030b0     LIBCMT:undname.obj
 0001:000020b8       ??_C@_09BLBHBJP@?$GAvbtable?8?$AA@ 100030b8     LIBCMT:undname.obj
 0001:000020c4       ??_C@_09IFPLHPGF@?$GAvftable?8?$AA@ 100030c4     LIBCMT:undname.obj
 0001:000020d0       ??_C@_02MHEGNOJ@?$FO?$DN?$AA@ 100030d0     LIBCMT:undname.obj
 0001:000020d4       ??_C@_02DHLNPPGH@?$HM?$DN?$AA@ 100030d4     LIBCMT:undname.obj
 0001:000020d8       ??_C@_02FGJGFEAB@?$CG?$DN?$AA@ 100030d8     LIBCMT:undname.obj
 0001:000020dc       ??_C@_03CDNPDDLA@?$DM?$DM?$DN?$AA@ 100030dc     LIBCMT:undname.obj
 0001:000020e0       ??_C@_03IKFCCPFF@?$DO?$DO?$DN?$AA@ 100030e0     LIBCMT:undname.obj
 0001:000020e4       ??_C@_02FENAOKFI@?$CF?$DN?$AA@ 100030e4     LIBCMT:undname.obj
 0001:000020e8       ??_C@_02FJEHGPIO@?1?$DN?$AA@ 100030e8     LIBCMT:undname.obj
 0001:000020ec       ??_C@_02FKMDLLOA@?9?$DN?$AA@ 100030ec     LIBCMT:undname.obj
 0001:000020f0       ??_C@_02FOEOMHFC@?$CL?$DN?$AA@ 100030f0     LIBCMT:undname.obj
 0001:000020f4       ??_C@_02FPIMKNGF@?$CK?$DN?$AA@ 100030f4     LIBCMT:undname.obj
 0001:000020f8       ??_C@_02NONPIBCD@?$HM?$HM?$AA@ 100030f8     LIBCMT:undname.obj
 0001:000020fc       ??_C@_02PPKAJPJL@?$CG?$CG?$AA@ 100030fc     LIBCMT:undname.obj
 0001:00002100       ??_C@_01DNKMNLPK@?$HM?$AA@ 10003100     LIBCMT:undname.obj
 0001:00002104       ??_C@_01JKBOJNNK@?$FO?$AA@ 10003104     LIBCMT:undname.obj
 0001:00002108       ??_C@_01PJKLJHI@?$HO?$AA@  10003108     LIBCMT:undname.obj
 0001:0000210c       ??_C@_02HCKGKOFO@?$CI?$CJ?$AA@ 1000310c     LIBCMT:undname.obj
 0001:00002110       ??_C@_01IHBHIGKO@?0?$AA@   10003110     LIBCMT:undname.obj
 0001:00002114       ??_C@_02EEKDKGMJ@?$DO?$DN?$AA@ 10003114     LIBCMT:undname.obj
 0001:00002118       ??_C@_01PPODPGHN@?$DO?$AA@ 10003118     LIBCMT:undname.obj
 0001:0000211c       ??_C@_02EHCHHCKH@?$DM?$DN?$AA@ 1000311c     LIBCMT:undname.obj
 0001:00002120       ??_C@_01MNNFJEPP@?$DM?$AA@ 10003120     LIBCMT:undname.obj
 0001:00002124       ??_C@_01FGNFDNOH@?$CF?$AA@ 10003124     LIBCMT:undname.obj
 0001:00002128       ??_C@_01KMDKNFGN@?1?$AA@   10003128     LIBCMT:undname.obj
 0001:0000212c       ??_C@_03MNHNFDLC@?9?$DO?$CK?$AA@ 1000312c     LIBCMT:undname.obj
 0001:00002130       ??_C@_01HNPIGOCE@?$CG?$AA@ 10003130     LIBCMT:undname.obj
 0001:00002134       ??_C@_01MIFGBAGJ@?$CL?$AA@ 10003134     LIBCMT:undname.obj
 0001:00002138       ??_C@_01JOAMLHOP@?9?$AA@   10003138     LIBCMT:undname.obj
 0001:0000213c       ??_C@_02BAABKJLB@?9?9?$AA@ 1000313c     LIBCMT:undname.obj
 0001:00002140       ??_C@_02ECNGHCIF@?$CL?$CL?$AA@ 10003140     LIBCMT:undname.obj
 0001:00002144       ??_C@_01NBENCBCI@?$CK?$AA@ 10003144     LIBCMT:undname.obj
 0001:00002148       ??_C@_02HBOOOICD@?9?$DO?$AA@ 10003148     LIBCMT:undname.obj
 0001:0000214c       ??_C@_08LHJFAFGD@operator?$AA@ 1000314c     LIBCMT:undname.obj
 0001:00002158       ??_C@_02GPECMEKF@?$FL?$FN?$AA@ 10003158     LIBCMT:undname.obj
 0001:0000215c       ??_C@_02FDNJECIE@?$CB?$DN?$AA@ 1000315c     LIBCMT:undname.obj
 0001:00002160       ??_C@_02EGOFBIJA@?$DN?$DN?$AA@ 10003160     LIBCMT:undname.obj
 0001:00002164       ??_C@_01DCLJPIOD@?$CB?$AA@ 10003164     LIBCMT:undname.obj
 0001:00002168       ??_C@_02FODMEDOG@?$DM?$DM?$AA@ 10003168     LIBCMT:undname.obj
 0001:0000216c       ??_C@_02GPIOPFAK@?$DO?$DO?$AA@ 1000316c     LIBCMT:undname.obj
 0001:00002170       ??_C@_07FPCDHGMM@?5delete?$AA@ 10003170     LIBCMT:undname.obj
 0001:00002178       ??_C@_04NIHEBCM@?5new?$AA@ 10003178     LIBCMT:undname.obj
 0001:00002180       ??_C@_0M@GFIIJFMG@__unaligned?$AA@ 10003180     LIBCMT:undname.obj
 0001:0000218c       ??_C@_0L@PILCLIHE@__restrict?$AA@ 1000318c     LIBCMT:undname.obj
 0001:00002198       ??_C@_07JOMMBBKO@__ptr64?$AA@ 10003198     LIBCMT:undname.obj
 0001:000021a0       ??_C@_06GHPCKEAG@__eabi?$AA@ 100031a0     LIBCMT:undname.obj
 0001:000021a8       ??_C@_09HIJEGCPM@__clrcall?$AA@ 100031a8     LIBCMT:undname.obj
 0001:000021b4       ??_C@_0L@JMKHOMEK@__fastcall?$AA@ 100031b4     LIBCMT:undname.obj
 0001:000021c0       ??_C@_0L@NPHFGOKO@__thiscall?$AA@ 100031c0     LIBCMT:undname.obj
 0001:000021cc       ??_C@_09IFJBGAPI@__stdcall?$AA@ 100031cc     LIBCMT:undname.obj
 0001:000021d8       ??_C@_08GHMPAG@__pascal?$AA@ 100031d8     LIBCMT:undname.obj
 0001:000021e4       ??_C@_07KOLFKCDI@__cdecl?$AA@ 100031e4     LIBCMT:undname.obj
 0001:000021ec       ??_C@_08EHJDFFNH@__based?$CI?$AA@ 100031ec     LIBCMT:undname.obj
 0001:00002380       __load_config_used         10003380     LIBCMT:loadcfg.obj
 0001:000023c8       ??_R4bad_alloc@std@@6B@    100033c8     LIBCMT:new.obj
 0001:000023dc       ??_R3bad_alloc@std@@8      100033dc     LIBCMT:new.obj
 0001:000023ec       ??_R2bad_alloc@std@@8      100033ec     LIBCMT:new.obj
 0001:000023f8       ??_R1A@?0A@EA@bad_alloc@std@@8 100033f8     LIBCMT:new.obj
 0001:00002414       ??_R1A@?0A@EA@exception@std@@8 10003414     LIBCMT:new.obj
 0001:00002430       ??_R3exception@std@@8      10003430     LIBCMT:new.obj
 0001:00002440       ??_R2exception@std@@8      10003440     LIBCMT:new.obj
 0001:00002448       ??_R4exception@std@@6B@    10003448     LIBCMT:stdexcpt.obj
 0001:0000245c       ??_R4type_info@@6B@        1000345c     LIBCMT:typinfo.obj
 0001:00002470       ??_R3type_info@@8          10003470     LIBCMT:typinfo.obj
 0001:00002480       ??_R2type_info@@8          10003480     LIBCMT:typinfo.obj
 0001:00002488       ??_R1A@?0A@EA@type_info@@8 10003488     LIBCMT:typinfo.obj
 0001:000024b0       ___safe_se_handler_table   100034b0     <linker-defined>
 0001:000024bc       ___rtc_iaa                 100034bc     LIBCMT:_initsect_.obj
 0001:000024c0       ___rtc_izz                 100034c0     LIBCMT:_initsect_.obj
 0001:000024c4       ___rtc_taa                 100034c4     LIBCMT:_initsect_.obj
 0001:000024c8       ___rtc_tzz                 100034c8     LIBCMT:_initsect_.obj
 0001:000024d0       __alloca_probe             100034d0     chkstk.obj
 0001:000024d0       __chkstk                   100034d0 f   chkstk.obj
 0001:00002500       ??0SimpleString@@QAE@PB_WI@Z 10003500 f i Compare.obj
 0001:00002580       ?Inflate@SimpleString@@QAEXI@Z 10003580 f i Compare.obj
 0001:00002720       ?ShowDialogProc@@YGHPAXHH0@Z 10003720 f   Compare.obj
 0001:00002fa0       ?BuildName@FileName@@QAEPB_WPB_W0@Z 10003fa0 f i Compare.obj
 0001:00003260       ?isnewline@@YA_NH@Z        10004260 f   Compare.obj
 0001:00003280       _GetGlobalInfoW@4          10004280 f   Compare.obj
 0001:00003300       _SetStartupInfoW@4         10004300 f   Compare.obj
 0001:00003330       _GetPluginInfoW@4          10004330 f   Compare.obj
 0001:00003370       ?GetPanelItem@@YAXPAXW4FILE_CONTROL_COMMANDS@@HPAUPluginPanelItem@@@Z 10004370 f   Compare.obj
 0001:00003410       ?FreePanelItems@@YAXAAUOwnPanelInfo@@0@Z 10004410 f   Compare.obj
 0001:00003510       ?Replace@SimpleString@@QAEAAV1@IIPB_WI@Z 10004510 f i Compare.obj
 0001:00003970       ??0SimpleString@@QAE@PB_W@Z 10004970 f i Compare.obj
 0001:00004670       _OpenW@4                   10005670 f   Compare.obj
 0001:00004e83       ??_U@YAPAXI@Z              10005e83 f   libcpmt:newaop.obj
 0001:00004e90       _memcpy                    10005e90 f   LIBCMT:memcpy.obj
 0001:00005200       _memmove                   10006200 f   LIBCMT:memmove.obj
 0001:00005561       _realloc                   10006561 f   LIBCMT:realloc.obj
 0001:0000560e       _free                      1000660e f   LIBCMT:free.obj
 0001:00005650       _memset                    10006650 f   LIBCMT:memset.obj
 0001:000056ca       _wcschr                    100066ca f   LIBCMT:wcschr.obj
 0001:000056f1       ??_V@YAXPAX@Z              100066f1 f   LIBCMT:delete2.obj
 0001:000056fc       _malloc                    100066fc f   LIBCMT:malloc.obj
 0001:00005790       ??0_LocaleUpdate@@QAE@PAUlocaleinfo_struct@@@Z 10006790 f i LIBCMT:_ctype.obj
 0001:00005817       __isspace_l                10006817 f i LIBCMT:_ctype.obj
 0001:00005868       _isspace                   10006868 f i LIBCMT:_ctype.obj
 0001:00005896       __CRT_INIT@12              10006896 f   LIBCMT:dllcrt0.obj
 0001:00005af0       __DllMainCRTStartup@12     10006af0 f   LIBCMT:dllcrt0.obj
 0001:00005b13       ??1bad_alloc@std@@UAE@XZ   10006b13 f i LIBCMT:new.obj
 0001:00005b1e       ??_Ebad_alloc@std@@UAEPAXI@Z 10006b1e f i LIBCMT:new.obj
 0001:00005b1e       ??_Gbad_alloc@std@@UAEPAXI@Z 10006b1e f i LIBCMT:new.obj
 0001:00005b45       ??0bad_alloc@std@@QAE@ABV01@@Z 10006b45 f i LIBCMT:new.obj
 0001:00005b62       ??2@YAPAXI@Z               10006b62 f   LIBCMT:new.obj
 0001:00005be2       __VEC_memcpy               10006be2 f   LIBCMT:p4_memcpy.obj
 0001:00005ce5       ___sse2_available_init     10006ce5 f   LIBCMT:cpu_disp.obj
 0001:00005cf5       __get_errno_from_oserr     10006cf5 f   LIBCMT:dosmap.obj
 0001:00005d37       __errno                    10006d37 f   LIBCMT:dosmap.obj
 0001:00005d4a       __initp_heap_handler       10006d4a f   LIBCMT:handler.obj
 0001:00005d59       __callnewh                 10006d59 f   LIBCMT:handler.obj
 0001:00005d81       __heap_init                10006d81 f   LIBCMT:heapinit.obj
 0001:00005d9f       __heap_term                10006d9f f   LIBCMT:heapinit.obj
 0001:00005db3       __VEC_memzero              10006db3 f   LIBCMT:p4_memset.obj
 0001:00005e6d       ??3@YAXPAX@Z               10006e6d f   LIBCMT:delete.obj
 0001:00005e78       ___crtCorExitProcess       10006e78 f   LIBCMT:crt0dat.obj
 0001:00005ea3       ___crtExitProcess          10006ea3 f   LIBCMT:crt0dat.obj
 0001:00005ebb       __lockexit                 10006ebb f   LIBCMT:crt0dat.obj
 0001:00005ec4       __unlockexit               10006ec4 f   LIBCMT:crt0dat.obj
 0001:00005ecd       __init_pointers            10006ecd f   LIBCMT:crt0dat.obj
 0001:00005f00       __initterm_e               10006f00 f   LIBCMT:crt0dat.obj
 0001:00005f24       __cinit                    10006f24 f   LIBCMT:crt0dat.obj
 0001:000060fb       __exit                     100070fb f   LIBCMT:crt0dat.obj
 0001:00006111       __cexit                    10007111 f   LIBCMT:crt0dat.obj
 0001:00006120       __amsg_exit                10007120 f   LIBCMT:crt0dat.obj
 0001:0000613e       __GET_RTERRMSG             1000713e f   LIBCMT:crt0msg.obj
 0001:00006164       __NMSG_WRITE               10007164 f   LIBCMT:crt0msg.obj
 0001:00006313       __FF_MSGBANNER             10007313 f   LIBCMT:crt0msg.obj
 0001:0000656f       ___updatetmbcinfo          1000756f f   LIBCMT:mbctype.obj
 0001:0000668f       __setmbcp_nolock           1000768f f   LIBCMT:mbctype.obj
 0001:00006878       __setmbcp                  10007878 f   LIBCMT:mbctype.obj
 0001:00006a12       ___initmbctable            10007a12 f   LIBCMT:mbctype.obj
 0001:00006a30       ___addlocaleref            10007a30 f   LIBCMT:localref.obj
 0001:00006abf       ___removelocaleref         10007abf f   LIBCMT:localref.obj
 0001:00006b58       ___freetlocinfo            10007b58 f   LIBCMT:localref.obj
 0001:00006ca3       __updatetlocinfoEx_nolock  10007ca3 f   LIBCMT:localref.obj
 0001:00006cf0       ___updatetlocinfo          10007cf0 f   LIBCMT:localref.obj
 0001:00006d69       __encoded_null             10007d69 f   LIBCMT:tidtable.obj
 0001:00006d72       ___crtTlsAlloc@4           10007d72 f   LIBCMT:tidtable.obj
 0001:00006d7b       ___set_flsgetvalue         10007d7b f   LIBCMT:tidtable.obj
 0001:00006daf       __mtterm                   10007daf f   LIBCMT:tidtable.obj
 0001:00006dec       __initptd                  10007dec f   LIBCMT:tidtable.obj
 0001:00006ea0       __getptd_noexit            10007ea0 f   LIBCMT:tidtable.obj
 0001:00006f19       __getptd                   10007f19 f   LIBCMT:tidtable.obj
 0001:00006f33       __freefls@4                10007f33 f   LIBCMT:tidtable.obj
 0001:00007062       __freeptd                  10008062 f   LIBCMT:tidtable.obj
 0001:000070d0       __mtinit                   100080d0 f   LIBCMT:tidtable.obj
 0001:0000724b       __isctype_l                1000824b f   LIBCMT:isctype.obj
 0001:00007303       __malloc_crt               10008303 f   LIBCMT:crtheap.obj
 0001:00007348       __calloc_crt               10008348 f   LIBCMT:crtheap.obj
 0001:00007394       __realloc_crt              10008394 f   LIBCMT:crtheap.obj
 0001:000073e2       __ioinit                   100083e2 f   LIBCMT:ioinit.obj
 0001:00007627       __ioterm                   10008627 f   LIBCMT:ioinit.obj
 0001:0000767a       __setenvp                  1000867a f   LIBCMT:stdenvp.obj
 0001:000078f0       __setargv                  100088f0 f   LIBCMT:stdargv.obj
 0001:000079ab       ___crtGetEnvironmentStringsA 100089ab f   LIBCMT:a_env.obj
 0001:00007a42       __RTC_Initialize           10008a42 f   LIBCMT:_initsect_.obj
 0001:00007a68       __RTC_Terminate            10008a68 f   LIBCMT:_initsect_.obj
 0001:00007a90       __SEH_prolog4              10008a90 f   LIBCMT:sehprolg4.obj
 0001:00007ad5       __SEH_epilog4              10008ad5 f   LIBCMT:sehprolg4.obj
 0001:00007af0       __except_handler4          10008af0 f   LIBCMT:chandler4.obj
 0001:00007c7f       __XcptFilter               10008c7f f   LIBCMT:winxfltr.obj
 0001:00007dc9       ___CppXcptFilter           10008dc9 f   LIBCMT:winxfltr.obj
 0001:00007de9       _DllMain@12                10008de9 f   LIBCMT:dllmain.obj
 0001:00007def       ___security_init_cookie    10008def f   LIBCMT:gs_support.obj
 0001:00007e8a       ??0exception@std@@QAE@ABQBDH@Z 10008e8a f   LIBCMT:stdexcpt.obj
 0001:00007ea7       ?what@exception@std@@UBEPBDXZ 10008ea7 f   LIBCMT:stdexcpt.obj
 0001:00007eb4       ?_Copy_str@exception@std@@AAEXPBD@Z 10008eb4 f   LIBCMT:stdexcpt.obj
 0001:00007ef4       ?_Tidy@exception@std@@AAEXXZ 10008ef4 f   LIBCMT:stdexcpt.obj
 0001:00007f12       ??4exception@std@@QAEAAV01@ABV01@@Z 10008f12 f   LIBCMT:stdexcpt.obj
 0001:00007f47       ??1exception@std@@UAE@XZ   10008f47 f   LIBCMT:stdexcpt.obj
 0001:00007f52       ??_Eexception@std@@UAEPAXI@Z 10008f52 f i LIBCMT:stdexcpt.obj
 0001:00007f52       ??_Gexception@std@@UAEPAXI@Z 10008f52 f i LIBCMT:stdexcpt.obj
 0001:00007f79       ??0exception@std@@QAE@ABV01@@Z 10008f79 f   LIBCMT:stdexcpt.obj
 0001:00007f9e       ??1type_info@@UAE@XZ       10008f9e f   LIBCMT:typinfo.obj
 0001:00007fae       ??_Etype_info@@UAEPAXI@Z   10008fae f i LIBCMT:typinfo.obj
 0001:00007fae       ??_Gtype_info@@UAEPAXI@Z   10008fae f i LIBCMT:typinfo.obj
 0001:00008085       ___onexitinit              10009085 f   LIBCMT:onexit.obj
 0001:000080b6       __onexit                   100090b6 f   LIBCMT:onexit.obj
 0001:000080f2       _atexit                    100090f2 f   LIBCMT:onexit.obj
 0001:00008109       __CxxThrowException@8      10009109 f   LIBCMT:throw.obj
 0001:00008155       __initp_misc_invarg        10009155 f   LIBCMT:invarg.obj
 0001:00008164       __call_reportfault         10009164 f   LIBCMT:invarg.obj
 0001:0000828d       __invoke_watson            1000928d f   LIBCMT:invarg.obj
 0001:000082b2       __invalid_parameter        100092b2 f   LIBCMT:invarg.obj
 0001:000082df       __invalid_parameter_noinfo 100092df f   LIBCMT:invarg.obj
 0001:000082ef       __mtinitlocks              100092ef f   LIBCMT:mlock.obj
 0001:00008339       __mtdeletelocks            10009339 f   LIBCMT:mlock.obj
 0001:00008390       __unlock                   10009390 f   LIBCMT:mlock.obj
 0001:000083a7       __mtinitlocknum            100093a7 f   LIBCMT:mlock.obj
 0001:00008469       __lock                     10009469 f   LIBCMT:mlock.obj
 0001:0000849c       ?terminate@@YAXXZ          1000949c f   LIBCMT:hooks.obj
 0001:000084d5       __initp_eh_hooks           100094d5 f   LIBCMT:hooks.obj
 0001:000084e6       __initp_misc_winsig        100094e6 f   LIBCMT:winsig.obj
 0001:0000853b       ___get_sigabrt             1000953b f   LIBCMT:winsig.obj
 0001:00008548       _raise                     10009548 f   LIBCMT:winsig.obj
 0001:000086eb       __initp_misc_rand_s        100096eb f   LIBCMT:rand_s.obj
 0001:000086fa       __initp_misc_purevirt      100096fa f   LIBCMT:inithelp.obj
 0001:00008709       __initp_misc_cfltcvt_tab   10009709 f   LIBCMT:cmiscdat.obj
 0001:00008730       __ValidateImageBase        10009730 f   LIBCMT:pesect.obj
 0001:00008770       __FindPESection            10009770 f   LIBCMT:pesect.obj
 0001:000087c0       __IsNonwritableInCurrentImage 100097c0 f   LIBCMT:pesect.obj
 0001:00008880       _strlen                    10009880 f   LIBCMT:strlen.obj
 0001:0000890b       ___crtMessageBoxW          1000990b f   LIBCMT:crtmboxw.obj
 0001:00008a77       _wcscat_s                  10009a77 f   LIBCMT:wcscat_s.obj
 0001:00008aec       _wcsncpy_s                 10009aec f   LIBCMT:wcsncpy_s.obj
 0001:00008bb9       _wcslen                    10009bb9 f   LIBCMT:wcslen.obj
 0001:00008bd4       _wcscpy_s                  10009bd4 f   LIBCMT:wcscpy_s.obj
 0001:00008c37       __set_error_mode           10009c37 f   LIBCMT:errmode.obj
 0001:00008c76       @__security_check_cookie@4 10009c76 f   LIBCMT:secchk.obj
 0001:00008c85       __freea                    10009c85 f i LIBCMT:a_map.obj
 0001:00008e8c       ___crtLCMapStringA         10009e8c f   LIBCMT:a_map.obj
 0001:00008fb9       ___crtGetStringTypeA       10009fb9 f   LIBCMT:a_str.obj
 0001:00008ff9       ___free_lc_time            10009ff9 f   LIBCMT:inittime.obj
 0001:00009370       ___free_lconv_num          1000a370 f   LIBCMT:initnum.obj
 0001:000093d9       ___free_lconv_mon          1000a3d9 f   LIBCMT:initmon.obj
 0001:000094d7       __isleadbyte_l             1000a4d7 f i LIBCMT:_wctype.obj
 0001:00009510       _strcspn                   1000a510 f   LIBCMT:strcspn.obj
 0001:00009556       _strcpy_s                  1000a556 f   LIBCMT:strcpy_s.obj
 0001:000095c0       _strcmp                    1000a5c0 f   LIBCMT:strcmp.obj
 0001:00009650       _strpbrk                   1000a650 f   LIBCMT:strpbrk.obj
 0001:00009690       __calloc_impl              1000a690 f   LIBCMT:calloc_impl.obj
 0001:00009765       __ismbblead                1000a765 f   LIBCMT:ismbbyte.obj
 0001:00009780       __local_unwind4            1000a780 f   LIBCMT:exsup4.obj
 0001:00009856       __seh_longjmp_unwind4@4    1000a856 f   LIBCMT:exsup4.obj
 0001:00009872       @_EH4_CallFilterFunc@8     1000a872 f   LIBCMT:exsup4.obj
 0001:00009889       @_EH4_TransferToHandler@8  1000a889 f   LIBCMT:exsup4.obj
 0001:000098a2       @_EH4_GlobalUnwind2@8      1000a8a2 f   LIBCMT:exsup4.obj
 0001:000098bb       @_EH4_LocalUnwind@16       1000a8bb f   LIBCMT:exsup4.obj
 0001:000098d2       ?_Type_info_dtor@type_info@@CAXPAV1@@Z 1000a8d2 f   LIBCMT:typname.obj
 0001:00009942       __msize                    1000a942 f   LIBCMT:msize.obj
 0001:00009975       __crt_debugger_hook        1000a975 f   LIBCMT:dbghook.obj
 0001:0000997d       _abort                     1000a97d f   LIBCMT:abort.obj
 0001:000099b0       __fptrap                   1000a9b0 f   LIBCMT:crt0fp.obj
 0001:000099b9       ___report_gsfailure        1000a9b9 f   LIBCMT:gs_report.obj
 0001:00009ac0       __alloca_probe_16          1000aac0 f   LIBCMT:alloca16.obj
 0001:00009ad6       __alloca_probe_8           1000aad6     LIBCMT:alloca16.obj
 0001:00009af0       __global_unwind2           1000aaf0 f   LIBCMT:exsup.obj
 0001:00009b55       __local_unwind2            1000ab55 f   LIBCMT:exsup.obj
 0001:00009bd9       __abnormal_termination     1000abd9 f   LIBCMT:exsup.obj
 0001:00009bfc       __NLG_Notify1              1000abfc f   LIBCMT:exsup.obj
 0001:00009c05       __NLG_Notify               1000ac05 f   LIBCMT:exsup.obj
 0001:00009c1c       __NLG_Dispatch2            1000ac1c     LIBCMT:exsup.obj
 0001:00009c1c       __NLG_Dispatch             1000ac1c     LIBCMT:exsup.obj
 0001:00009c24       __NLG_Call                 1000ac24 f   LIBCMT:exsup.obj
 0001:00009c26       __NLG_Return2              1000ac26     LIBCMT:exsup.obj
 0001:00009c30       ___ascii_strnicmp          1000ac30 f   LIBCMT:_strnicm.obj
 0001:00009ca0       __aulldvrm                 1000aca0 f   LIBCMT:ulldvrm.obj
 0001:00009d40       __allmul                   1000ad40 f   LIBCMT:llmul.obj
 0001:00009d74       _RtlUnwind@16              1000ad74 f   kernel32:KERNEL32.dll
 0001:00009d7a       _wcsdup                    1000ad7a f   LIBCMT:wcsdup.obj
 0001:00009d7a       __wcsdup                   1000ad7a f   LIBCMT:wcsdup.obj
 0001:00009dcf       _calloc                    1000adcf f   LIBCMT:calloc.obj
 0001:00009e64       __TI2?AVbad_alloc@std@@    1000ae64     LIBCMT:new.obj
 0001:00009e74       __CTA2?AVbad_alloc@std@@   1000ae74     LIBCMT:new.obj
 0001:00009e80       __CT??_R0?AVbad_alloc@std@@@8??0bad_alloc@std@@QAE@ABV01@@Z12 1000ae80     LIBCMT:new.obj
 0001:00009e9c       __CT??_R0?AVexception@std@@@8??0exception@std@@QAE@ABV01@@Z12 1000ae9c     LIBCMT:new.obj
 0001:0000a044       __IMPORT_DESCRIPTOR_KERNEL32 1000b044     kernel32:KERNEL32.dll
 0001:0000a058       __NULL_IMPORT_DESCRIPTOR   1000b058     kernel32:KERNEL32.dll
 0002:00000260       ??_R0?AVbad_alloc@std@@@8  1000c260     LIBCMT:new.obj
 0002:0000027c       ??_R0?AVexception@std@@@8  1000c27c     LIBCMT:new.obj
 0002:00000408       ___initialmbcinfo          1000c408     LIBCMT:mbctype.obj
 0002:00000628       __mbctype                  1000c628     LIBCMT:mbctype.obj
 0002:00000730       __mbcasemap                1000c730     LIBCMT:mbctype.obj
 0002:00000830       ___ptmbcinfo               1000c830     LIBCMT:mbctype.obj
 0002:00000928       ___globallocalestatus      1000c928     LIBCMT:glstatus.obj
 0002:0000092c       ___clocalestr              1000c92c     LIBCMT:nlsdata2.obj
 0002:00000930       ___lc_time_c               1000c930     LIBCMT:nlsdata2.obj
 0002:00000a98       ___initiallocinfo          1000ca98     LIBCMT:nlsdata2.obj
 0002:00000b70       ___ptlocinfo               1000cb70     LIBCMT:nlsdata2.obj
 0002:00000b74       ___flsindex                1000cb74     LIBCMT:tidtable.obj
 0002:00000b78       ___getvalueindex           1000cb78     LIBCMT:tidtable.obj
 0002:00000b80       ___badioinfo               1000cb80     LIBCMT:ioinit.obj
 0002:00000bc0       ??_R0?AVtype_info@@@8      1000cbc0     LIBCMT:typinfo.obj
 0002:00000cf8       __cfltcvt_tab              1000ccf8     LIBCMT:cmiscdat.obj
 0002:00000d20       ___security_cookie         1000cd20     LIBCMT:gs_cookie.obj
 0002:00000d24       ___security_cookie_complement 1000cd24     LIBCMT:gs_cookie.obj
 0002:00000d28       ___lconv_static_decimal    1000cd28     LIBCMT:lconv.obj
 0002:00000d2c       ___lconv_static_W_decimal  1000cd2c     LIBCMT:lconv.obj
 0002:00000d30       ___lconv_c                 1000cd30     LIBCMT:lconv.obj
 0002:00000d80       ___lconv                   1000cd80     LIBCMT:lconv.obj
 0002:00000d84       __pctype                   1000cd84     LIBCMT:ctype.obj
 0002:00000d88       __pwctype                  1000cd88     LIBCMT:ctype.obj
 0002:00000d8c       ___mb_cur_max              1000cd8c     LIBCMT:nlsdata1.obj
 0002:00000d90       ___decimal_point           1000cd90     LIBCMT:nlsdata1.obj
 0002:00000d94       ___decimal_point_length    1000cd94     LIBCMT:nlsdata1.obj
 0002:00000da0       ___abort_behavior          1000cda0     LIBCMT:abort.obj
 0002:00000db0       __NLG_Destination          1000cdb0     LIBCMT:exsup.obj
 0002:00000f28       ?Opt@@3UOptions@@A         1000cf28     Compare.obj
 0002:00000f80       __aenvptr                  1000cf80     LIBCMT:dllcrt0.obj
 0002:00000f84       __wenvptr                  1000cf84     LIBCMT:dllcrt0.obj
 0002:00000f88       ___error_mode              1000cf88     LIBCMT:dllcrt0.obj
 0002:00000f8c       ___app_type                1000cf8c     LIBCMT:dllcrt0.obj
 0002:00000fa0       ?_pnhHeap@@3P6AHI@ZA       1000cfa0     LIBCMT:handler.obj
 0002:00000fa4       __newmode                  1000cfa4     LIBCMT:_newmode.obj
 0002:00000fa8       __crtheap                  1000cfa8     LIBCMT:heapinit.obj
 0002:00000fac       __umaskval                 1000cfac     LIBCMT:crt0dat.obj
 0002:00000fb0       ___argc                    1000cfb0     LIBCMT:crt0dat.obj
 0002:00000fb4       ___argv                    1000cfb4     LIBCMT:crt0dat.obj
 0002:00000fb8       ___wargv                   1000cfb8     LIBCMT:crt0dat.obj
 0002:00000fbc       __environ                  1000cfbc     LIBCMT:crt0dat.obj
 0002:00000fc0       ___initenv                 1000cfc0     LIBCMT:crt0dat.obj
 0002:00000fc4       __wenviron                 1000cfc4     LIBCMT:crt0dat.obj
 0002:00000fc8       ___winitenv                1000cfc8     LIBCMT:crt0dat.obj
 0002:00000fcc       __pgmptr                   1000cfcc     LIBCMT:crt0dat.obj
 0002:00000fd0       __wpgmptr                  1000cfd0     LIBCMT:crt0dat.obj
 0002:00000fd4       __exitflag                 1000cfd4     LIBCMT:crt0dat.obj
 0002:00000fd8       __C_Termination_Done       1000cfd8     LIBCMT:crt0dat.obj
 0002:00000fdc       __C_Exit_Done              1000cfdc     LIBCMT:crt0dat.obj
 0002:0000160c       ___mbulinfo                1000d60c     LIBCMT:mbctype.obj
 0002:00001618       ___mbcodepage              1000d618     LIBCMT:mbctype.obj
 0002:0000161c       ___ismbcodepage            1000d61c     LIBCMT:mbctype.obj
 0002:00001620       ___mblcid                  1000d620     LIBCMT:mbctype.obj
 0002:00001624       _gpFlsAlloc                1000d624     LIBCMT:tidtable.obj
 0002:00001628       _gpFlsGetValue             1000d628     LIBCMT:tidtable.obj
 0002:0000162c       _gpFlsSetValue             1000d62c     LIBCMT:tidtable.obj
 0002:00001630       _gpFlsFree                 1000d630     LIBCMT:tidtable.obj
 0002:00001634       ___locale_changed          1000d634     LIBCMT:setlocal.obj
 0002:00001638       __maxwait                  1000d638     LIBCMT:crtheap.obj
 0002:00001748       ___pInvalidArgHandler      1000d748     LIBCMT:invarg.obj
 0002:000018a0       ?__pInconsistency@@3P6AXXZA 1000d8a0     LIBCMT:hooks.obj
 0002:000018bc       ___pPurecall               1000d8bc     LIBCMT:inithelp.obj
 0002:000018d4       ___lconv_static_null       1000d8d4     LIBCMT:lconv.obj
 0002:000018d8       ___lconv_static_W_null     1000d8d8     LIBCMT:lconv.obj
 0002:00001c20       ?pArgList@UnDecorator@@0PAVReplicator@@A 1000dc20     LIBCMT:undname.obj
 0002:00001c24       ?pZNameList@UnDecorator@@0PAVReplicator@@A 1000dc24     LIBCMT:undname.obj
 0002:00001c28       ?pTemplateArgList@UnDecorator@@0PAVReplicator@@A 1000dc28     LIBCMT:undname.obj
 0002:00001c2c       ?gName@UnDecorator@@0PBDB  1000dc2c     LIBCMT:undname.obj
 0002:00001c30       ?name@UnDecorator@@0PBDB   1000dc30     LIBCMT:undname.obj
 0002:00001c34       ?outputString@UnDecorator@@0PADA 1000dc34     LIBCMT:undname.obj
 0002:00001c38       ?maxStringLength@UnDecorator@@0HA 1000dc38     LIBCMT:undname.obj
 0002:00001c3c       ?disableFlags@UnDecorator@@0KA 1000dc3c     LIBCMT:undname.obj
 0002:00001c40       ?m_pGetParameter@UnDecorator@@0P6APADJ@ZA 1000dc40     LIBCMT:undname.obj
 0002:00001c44       ?fExplicitTemplateParams@UnDecorator@@0_NA 1000dc44     LIBCMT:undname.obj
 0002:00001c45       ?fGetTemplateArgumentList@UnDecorator@@0_NA 1000dc45     LIBCMT:undname.obj
 0002:00001c48       __debugger_hook_dummy      1000dc48     <common>
 0002:00001c4c       __pDestructExceptionObject 1000dc4c     <common>
 0002:00001c50       __nhandle                  1000dc50     <common>
 0002:00001c60       ___pioinfo                 1000dc60     <common>
 0002:00001d60       ___env_initialized         1000dd60     <common>
 0002:00001d64       ___onexitend               1000dd64     <common>
 0002:00001d68       ___onexitbegin             1000dd68     <common>
 0002:00001d6c       ___mbctype_initialized     1000dd6c     <common>
 0002:00001d70       __FPinit                   1000dd70     <common>
 0002:00001d74       ___dyn_tls_init_callback   1000dd74     <common>
 0002:00001d78       ___sse2_available          1000dd78     <common>
 0002:00001d7c       __acmdln                   1000dd7c     <common>

 entry point at        0001:00005af0

 Static symbols

 0001:000025f0       ?WFD2FFD@@YAXAAU_WIN32_FIND_DATAW@@AAUPluginPanelItem@@@Z 100035f0 f   Compare.obj
 0001:00002660       ?GetSetting@@YA_JW4FARSETTINGS_SUBFOLDERS@@PB_W@Z 10003660 f   Compare.obj
 0001:00002860       ?ShowDialog@@YA_N_N0@Z     10003860 f   Compare.obj
 0001:00002e50       ?CheckForEsc@@YA_NXZ       10003e50 f   Compare.obj
 0001:00003070       ?PICompare@@YGHPBX0PAX@Z   10004070 f   Compare.obj
 0001:000030b0       ?BuildPanelIndex@@YA_NPBUOwnPanelInfo@@PAUFileIndex@@PAX@Z 100040b0 f   Compare.obj
 0001:00003210       ?FreeDirList@@YAXPAUOwnPanelInfo@@@Z 10004210 f   Compare.obj
 0001:00003620       ?SplitCopy@@YAHQAPA_WHPA_WPB_W@Z 10004620 f   Compare.obj
 0001:000037f0       ?ShowMessage@@YAXPB_W0@Z   100047f0 f   Compare.obj
 0001:00003a00       ?GetDirList@@YAHPAUOwnPanelInfo@@PB_W@Z 10004a00 f   Compare.obj
 0001:00003b40       ?CompareFiles@@YA_NPBUPluginPanelItem@@0PB_W1H@Z 10004b40 f   Compare.obj
 0001:00004300       ?CompareDirs@@YA_NPBUOwnPanelInfo@@0_NH@Z 10005300 f   Compare.obj
 0001:000059fa       ___DllMainCRTStartup       100069fa f   LIBCMT:dllcrt0.obj
 0001:00005fbb       _doexit                    10006fbb f   LIBCMT:crt0dat.obj
 0001:0000634c       ?CPtoLCID@@YAHH@Z          1000734c f   LIBCMT:mbctype.obj
 0001:0000637b       ?setSBCS@@YAXPAUthreadmbcinfostruct@@@Z 1000737b f   LIBCMT:mbctype.obj
 0001:000063df       ?setSBUpLow@@YAXPAUthreadmbcinfostruct@@@Z 100073df f   LIBCMT:mbctype.obj
 0001:00006613       ?getSystemCP@@YAHH@Z       10007613 f   LIBCMT:mbctype.obj
 0001:00007756       _parse_cmdline             10008756 f   LIBCMT:stdargv.obj
 0001:00007fcf       __onexit_nolock            10008fcf f   LIBCMT:onexit.obj
 0001:00008504       _siglookup                 10009504 f   LIBCMT:winsig.obj
 0001:00008ca5       ?__crtLCMapStringA_stat@@YAHPAUlocaleinfo_struct@@KKPBDHPADHHH@Z 10009ca5 f   LIBCMT:a_map.obj
 0001:00008ed2       ?__crtGetStringTypeA_stat@@YAHPAUlocaleinfo_struct@@KPBDHPAGHHH@Z 10009ed2 f   LIBCMT:a_str.obj
 0001:00009712       ?x_ismbbtype_l@@YAHPAUlocaleinfo_struct@@IHH@Z 1000a712 f   LIBCMT:ismbbyte.obj
 0001:00009810       __unwind_handler4          1000a810 f   LIBCMT:exsup4.obj
 0001:00009b10       __unwind_handler           1000ab10 f   LIBCMT:exsup.obj
 0001:00009e0f       ??__Fnomem@?5???2@YAPAXI@Z@YAXXZ 1000ae0f f   LIBCMT:new.obj
